:080000000C9477000C94000041
:100008000C9400000C9400000C9400000C94000068
:100018000C9400000C9400000C9400000C94000058
:100028000C9400000C9400000C9400000C94000048
:100038000C9400000C9400000C9400000C94000038
:100048000C9400000C9400000C9400000C94000028
:100058000C9400000C94B5000C9400000C94000063
:100068000C9400000C9400000C9400000C94000008
:100078000C9400000C9400000C9400000C940000F8
:100088000C9400000C9400000C9400000C940000E8
:100098000C9400000C9400000C9400000C940000D8
:1000A8000C9400000C9400000C9400000C940000C8
:1000B8000C9400000C9400000C9400000C940000B8
:1000C8000C9400000C9400000C9400000C940000A8
:1000D8000C9400000C9400000C9400000000010037
:1000E8000500E4000000F894EE27EFBBF1E0F5BF4F
:1000F800E5BFE0937400E0937500F8E1A895A4B714
:10010800A77FA4BFF0936000E09360008DE0A2E0B9
:10011800BB27ED938A95E9F780E090E2A0E0B2E092
:10012800ED930197E9F7E6EEF0E085919591009758
:1001380061F0A591B59105901590BF01F00105906A
:100148000D920197E1F7FB01F0CF8BBF8CBFE0E088
:10015800EEBBEFEFEDBFE1E2EEBFC0E0D6E00C94FE
:1001680014016A937A93AA93BA93EA93FA93EFB72E
:10017800EA93A2E0B6E0ED91FD913196FE93EE93FD
:10018800A0E0B6E0ED91FD913196FE93EE93A0913B
:100198000206B0910306A032EEE4BE0729F4E6E0B9
:1001A800F0E060E070E05E2EA0910206B0910306D8
:1001B800A034ECE9BE0751F4E7E1F0E060E070E05C
:1001C8005E2EE0E0E0930206E0930306E52DA091A1
:1001D8000006B0910106F0E0EA17FB0721F4289821
:1001E80029982A982B98A0910006B0910106A83C5E
:1001F800E0E0BE0749F4289A299A2A9A2B9AE0E067
:10020800E0930006E0930106E6B5E951E6BDE99101
:10021800EFBFF991E991B991A991799169911895EF
:10022800E0E0E5B9EFEFE4B9E0E0E4BDE3E0E5BD27
:10023800E7EEE6BDE1E0E0936E007894FFCFFFCFF4
:00000001FF
